:0600000088310028000019
:0800080083018A012000770842
:10001000A0007808A1007908A2007A08A3008B1E2E
:1000200013280B191C282008F7002108F8002208C3
:10003000F9002308FA00090080317F2902302100ED
:10004000C502031C3028203085007530840000086C
:10005000031930282E282C282D280000800B2B284F
:10006000200008002100C80148080F3C031CA728F5
:10007000C701C9014908073C031C9C28C601460862
:10008000C50020000C18522821004508133C031815
:100090004B2820005228C50A8530F700F70B4E2860
:1000A0004128200021004508143C031D6C28490804
:1000B000033C031869282730480784002030850056
:1000C0000318850A4708800001304807F800A9286E
:1000D0006C284808F800A92820000C1C7D28210065
:1000E00046089F3C0318762820007D28C60A8530E4
:1000F000F700F70B79286C28200021004608A03C67
:10010000031D8F28273048078400203085000318FE
:10011000850A4708800001304807F800A9284508EB
:10012000C5070310C70D4608450203189928471450
:100130009A284710C90A3A282730480784002030F7
:1001400085000318850A47088000C80A3428480833
:10015000F800200008002100C80148080F3C031CDB
:100160001629C701C9014908073C031C0B29C60110
:100170004608C50020000C18CB2821004508313C5A
:100180000318C4282000CB28C50A8530F700F70BD8
:10019000C728BA28200021004508323C031DDD286D
:1001A000273048078400203085000318850A470857
:1001B000800001304807F800182920000C1CEE28A8
:1001C00021004608133C0318E7282000EE28C60A41
:1001D0008530F700F70BEA28DD28200021004608CB
:1001E000143C031D00292730480784002030850077
:1001F0000318850A4708800001304807F8001829CD
:100200000310C70D45080F3C031C08294710092996
:100210004714C90AB32827304807840020308500D6
:100220000318850A47088000C80AAD284808F80066
:100230002000080021000C1420000C1C2229003092
:10024000F8007D292100C20120000C18342921006A
:100250004208773C03182E2920003429C20A643052
:10026000C50020001E20252921004208783C031DDE
:100270003E290030F80020007D292100C201200025
:100280000C1C502921004208773C03184929200002
:100290005029C20A8530F700F70B4C293F2920006E
:1002A00021004208783C031D5A290030F800200044
:1002B0007D2921004208143C0318662901302000E2
:1002C000D800322078082100C3006D2903302000B7
:1002D000D800AB2078082100C300C30803197B298C
:1002E00042083C3C031C7B294208133C031C7A292E
:1002F000C3177B2943174308F80020000800220099
:100300008C158C118B1220001A2178082100C00056
:10031000C0080319442A4008C20042083F39C500FA
:10032000C3014308013C031CCC290530430784006A
:10033000203085000318850A45080002031DCA29DC
:10034000C4014408C600450844020318C2292730E6
:1003500044078400203085000318850A0008C70080
:10036000430EF700F030F70577084407073E840096
:10037000203085000318850A00084702031DC229A2
:10038000C40AA32945084402031DCA2901304307B2
:10039000F800CE29C30A91290030F8007808BC0083
:1003A000BC080319442A3C08013A20000319DC293F
:1003B000033A03190D2A3E2AE208031DE6296108C3
:1003C000C73C031CE629E30A0319E40AE201E10140
:1003D000E408031DEF296308143C0318FD2958089D
:1003E000033C031DF82902302100C100FB29200035
:1003F00005302100C100002A200001302100C10089
:100400004108C103003A03190C2A200059087F3C17
:10041000031DD90A2100002A402AE208031D172AD9
:100420006108C73C031C172AE30A0319E40AE20126
:10043000E101E408031D202A6308143C03182E2A56
:100440005808033C031D292A04302100C1002C2A2E
:1004500020000A302100C100312A20000130210093
:10046000C1004108C103003A03193C2A2000D90801
:10047000031DD9032100312A402A20002100402AEF
:100480003C082000E70021008B1620006108FA3CA0
:10049000031D4D2AE2080319512AE10A0319E20A51
:1004A000532AE401E3012100BC0120008D1D5B2AD9
:1004B0002100BC0A20002100BD0120008D1C632A00
:1004C0002100BD0A2000DA080319042B2100BC0812
:1004D00003196C2A2000042B2000DE01DD0121001D
:1004E000BD080319792A2000DB0A0319DC0A7E2AD9
:1004F000210020005B080319DC03DB0321003C081A
:100500002000DA00E008031D032B5F08313C031CC8
:10051000032BDF08031D8F2AE0080319032B21009A
:10052000C3013230C200200060082100C500200055
:100530005F082100C400F801F901F701FA0145083C
:10054000031DA52A44080319BF2A1030C600031052
:10055000C20DC30DF70DFA0D45087A02031DB22A2C
:1005600044087702031CBB2A4408F702031CFA0361
:100570004508FA020314F80DF90DC60BA72A7808EE
:10058000BE00043C0318C62A0430BE0020005C08EC
:100590002100C30020005B082100C200C5013E0805
:1005A000C400430845068039C700C31FDC2AC209BE
:1005B000C309C20A0319C30AC51FE32AC409C5092E
:1005C000C40A0319C50A1030C600F701FA01C30CAA
:1005D000C20C031CF12A4408F7070318FA0A45085D
:1005E000FA07FA0CF70CF90CF80CC60BE72AC71F30
:1005F000FE2AF809F909F80A0319F90A790820000E
:10060000DC007808DB00122B21003C082000DA0017
:100610005F082C3C031D0F2B600B0F2B122BDF0AE6
:100620000319E00ADC1B282BDC08031D1B2B5B08CD
:10063000003C0318282B5B085C040319272B5B087C
:100640000319DC03DB03D908031DD9031B2B362B4D
:10065000DC1F362B5B085C040319362BDB0A0319FD
:10066000DC0A59087F3C031DD90A2A2BE508031D23
:100670003C2BE6080319402B65080319E603E50344
:100680000B118031132821008C1322008C172100BC
:100690000C1322000C1321008D130D1222000D12D9
:1006A00021008D1222008D16883120003A2820303A
:1006B000850063308400000803196B2B0A30F800B2
:1006C000F701F70B612BF80B602B5F30F700F70B8E
:1006D000672B800B5E2B080022008C132000EF0894
:1006E0000319762B22008D17782B200022008D1302
:1006F0000C170C138D170C170C130C170C130C176D
:100700000C130039F700210021080839FA00770896
:100710007A0403198F2B22008D17912B21002200C0
:100720008D130C170C130039F70021002108043930
:10073000FA0077087A040319A12B22008D17A32B46
:10074000210022008D130C170C130039F700210033
:1007500021080239FA0077087A040319B32B220022
:100760008D17B52B210022008D130C170C130039A7
:10077000F700210021080139FA0077087A040319EB
:10078000C52B22008D17C72B210022008D130C17BB
:100790000C13210020088039F700FA0177087A0449
:1007A0000319D62B22008D17D82B210022008D1380
:1007B0000C170C13210020084039F700FA017708C4
:1007C0007A040319E72B22008D17E92B2100220060
:1007D0008D130C170C13210020082039F700FA01A3
:1007E00077087A040319F82B22008D17FA2B2100C1
:1007F00022008D130C170C13210020081039F7006C
:10080000FA0177087A040319092C22008D170B2CA2
:10081000210022008D130C170C1321002008083929
:10082000F700FA0177087A0403191A2C22008D17B1
:100830001C2C210022008D130C170C132100200802
:100840000439F700FA0177087A0403192B2C2200E7
:100850008D172D2C210022008D130C170C13210055
:1008600020080239F700FA0177087A0403193C2CB2
:1008700022008D173E2C210022008D130C170C1323
:10088000210020080139F700FA0177087A040319DA
:100890004D2C22008D174F2C210022008D130C1798
:1008A0000C138C170D121A30F700F70B552C0000A3
:1008B0000D161A30F700F70B5B2C00002000080023
:1008C000EC01230091019513151413084F3C0319F3
:1008D0006C2C2000EC0A23000130910095131514B4
:1008E00013084B3C0319772C2000EC0A230002303C
:1008F0009100951315141308493C0319822C20000C
:10090000EC0A230003309100951315141308523C90
:1009100003198D2C2000EC0A23000430910095135C
:1009200015141308413C0319982C2000EC0A2300ED
:10093000053091009513151413084B3C0319A32C93
:100940002000EC0A230006309100951315141308BB
:10095000553C0319AE2C2000EC0A23002000ED01C9
:100960008D18ED0AEE018D19EE0A01302100B30059
:10097000200057232100A201A1012208033C031CEF
:10098000EF2C031DC72C2108833C031CEF2C2000F7
:10099000EF018D18EF0A2100A00120008D1DD32C3E
:1009A0002100A00A20006F086D020319DA2CEC0A5E
:1009B0006F08ED002100200820006E020319E52CCD
:1009C000EC0A210020082000EE0001302100B300D5
:1009D000200057232100A10A0319A20ABD2C2000E0
:1009E0006C08F80088314C28230091014F309300A7
:1009F000951315150B08F7008B1355309600AA3088
:100A0000960095149518022D151177088B04013066
:100A100091004B309300951315150B08F7008B13BD
:100A200055309600AA30960095149518152D15117D
:100A300077088B0402309100493093009513151507
:100A40000B08F7008B1355309600AA3096009514CA
:100A50009518282D151177088B040330910052301A
:100A60009300951315150B08F7008B13553096005E
:100A7000AA309600951495183B2D151177088B0414
:100A80000430910041309300951315150B08F700C1
:100A90008B1355309600AA309600951495184E2D5C
:100AA000151177088B04053091004B309300951396
:100AB00015150B08F7008B1355309600AA309600D9
:100AC00095149518612D151177088B040630910047
:100AD00055309300951315150B08F7008B135530FF
:100AE0009600AA30960095149518742D1511770864
:100AF0008B042000D90109302300910020005908FF
:100B000023009300951315150B08F7008B13553030
:100B10009600AA309600951495188C2D151177081B
:100B20008B042000ED01EC01ED08031DCA2D6C08BB
:100B3000013C031CCA2D10306C072100A2000030BC
:100B400020006D3D2100A300053020006C078400CB
:100B500020306D3D8500083080002100A40022086F
:100B600023009100210024082300930095131515FC
:100B70000B08F7008B1355309600AA309600951499
:100B80009518C02D151177088B042000EC0A031965
:100B9000ED0A942D2100A101A0012000ED01EC013E
:100BA000ED08031D082E6C08013C031C082EEF0104
:100BB000EE01EF08031D042E6E080F3C031C042EEB
:100BC000203021002007A2000030213DA300220890
:100BD0002300910055309300951315150B08F7006D
:100BE0008B1355309600AA30960095149518F62D63
:100BF000151177088B042100A00A0319A10A20000F
:100C0000EE0A0319EF0AD92DEC0A0319ED0AD02DCB
:100C10008831522822008C152000EF016F08013C1A
:100C2000031CC12E6F0B172E22000C152000A401EF
:100C30008B1BA4178B131A21A41B8B177808210078
:100C4000A000A008031D272E2000172E2100200041
:100C5000EC016C080F3C031C4D2E52306C07F80061
:100C60002030FA000318FA0A78082100B2007A0846
:100C7000B300273020006C07840020308500031863
:100C8000850A00082100B40033088500320884007A
:100C9000340880002000EC0A292E02302100B20026
:100CA000FA30B300200057232100B20B502E3F3002
:100CB000A005103020006F072100B2000530200091
:100CC0006F078400203085000318850A2100200862
:100CD00080002008B3003208230091002100200882
:100CE00023009300951315150B08F7008B1355304F
:100CF0009600AA309600951495187C2E1511770849
:100D00008B042000EC016C080F3C031CB42E6F0E0A
:100D1000F700F030F70577086C07203E2100B2009D
:100D2000523020006C078400203085000318850AAB
:100D300000082100B300320823009100210033088D
:100D400023009300951315150B08F7008B135530EE
:100D50009600AA30960095149518AC2E15117708B8
:100D60008B042000EC0A832E02302100B200FA30FE
:100D7000B300200057232100B20BB72E2000EF0A4A
:100D80000E2E22008C110C118831200055280930BC
:100D9000230091009513151413082000D900210099
:100DA000A101A0012000ED01EC01ED08031D352F8C
:100DB0006C08013C031C352F05306C078400203083
:100DC0006D3D850010306C072100A400003020002C
:100DD0006D3D2100A50024082300910095131514F2
:100DE000130880002000EF01EE01EF08031D312FF2
:100DF0006E080F3C031C312F6C0D2100A200200057
:100E00006D0D2100A300A20DA30DA20DA30DA20D37
:100E1000A30DF030A20520006E0821002207F80083
:100E200020006F082100233DFA007808073E840067
:100E300020307A3D850020302007A4000030213D7D
:100E4000A5002408230091009513151413088000B1
:100E50002100A00A0319A10A2000EE0A0319EF0AD3
:100E6000F52EEC0A0319ED0AD52E2100A101A001EF
:100E70002000ED01EC01ED08031D562F6C08013C2C
:100E8000031C562F05306C07840020306D3D850013
:100E900000087F39103C0318522F2100A00A0319C3
:100EA000A10A2000EC0A0319ED0A3B2F21002008BB
:100EB000F800883120005828EE016C08ED00ED0D97
:100EC000EE0DED0DEE0DED0DEE0DED0DEE0DED0D4E
:100ED000EE0DE030ED056C087F3C031D732F0F30E5
:100EE000EE00FF30ED00EF016E082100A1002000B0
:100EF0006D082100A00020006C230800E508031DF8
:100F0000A92FE608031DA92F1330E6008830E5005D
:100F10005908230091009513151413082000590255
:100F20000319A92F0930230091002000590823003C
:100F30009300951315150B08F7008B135530960089
:100F4000AA30960095149518A32F151177088B04D5
:060F500020008831AF28EB
:10100000850184011F308305F43021009900200000
:10101000D901DA01DC01DB01DE01DD01E001DF01E4
:10102000E201E101E401E3011330E6008830E5006C
:1010300023008C018D012200920191019401930102
:101040002000E701F03021009900FF308C008D0076
:1010500024008D00210095130D1122000D11210097
:101060008C1122008C1121000C1122000C118031F6
:101070002000432B883164302100B30080312000F0
:1010800057238831EF012100A101A0018031200008
:101090006C2388318031602C8831F8080319562878
:1010A0008031F42C883180310A2E88318031C72E6E
:1010B00088315908EC0080315C27883121001508FF
:1010C000C039043895000730200095008B16C030D9
:1010D0008B04E801680859020319AD285908680211
:1010E000031890286808590203198F28E80A68082D
:1010F000EC0080315C2788315808033C031D8828A8
:1011000005302100B30080312000572388318F281B
:1011100008302100B3008031200057238831AD28EA
:10112000680859020319AD28E8036808EC0080310B
:101130005C2788315808033C031DA6280530210090
:10114000B3008031200057238831AD2808302100BA
:10115000B300803120005723883180317E2F8831C1
:041160006A28630096
:020000040001F9
:04000E000439FF1E94
:00000001FF
